
Hexadecimal

Area                               Addr   Size   Decimal Bytes (Attributes)
--------------------------------   ----   ----   ------- ----- ------------
.  .ABS.                           0000   0000 =      0. bytes (ABS,CON)

      Value  Global
   --------  --------------------------------
     0000    l__CABS
     0000    l__GSINIT
     0000    l__HEAP
     0000    l__HOME
     0000    l__OVERLAY
     0000    s__HEADER
     0001    l__GSFINAL
     0002    l__DATA
     0006    l__HEADER
     0006    s__CODE
     0231    l__CODE
     0237    s__DATA
     0239    s__GSFINAL
     0239    s__GSINIT
     0239    s__HOME
     0239    s__OVERLAY
     023A    s__CABS
     023A    s__HEAP

Hexadecimal

Area                               Addr   Size   Decimal Bytes (Attributes)
--------------------------------   ----   ----   ------- ----- ------------
_CODE                              0006   0231 =    561. bytes (REL,CON)

      Value  Global
   --------  --------------------------------
     0006    _DOS
     0006    _DOS_start
     002D    _DOS_end
     002D    _main
     002D    _main_start
     0045    _main_end
     0053    _memset
     0053    _memset_start
     0069    _memcpy
     0069    _memcpy_start
     007E    _border
     007E    _border_start
     0093    _vsync
     0093    _vsync_start
     0095    _joystick
     0095    _joystick_start
     0098    _keyboard
     0098    _keyboard_start
     00A2    _mouse_pos
     00A2    _mouse_pos_start
     00BA    _mouse_set
     00BA    _mouse_set_start
     00CA    _mouse_clip
     00CA    _mouse_clip_start
     00E4    _mouse_delta
     00E4    _mouse_delta_start
     00FC    _sfx_play
     00FC    _sfx_play_start
     0106    _sfx_stop
     0106    _sfx_stop_start
     0109    _music_play
     0109    _music_play_start
     0111    _music_stop
     0111    _music_stop_start
     0114    _sample_play
     0114    _sample_play_start
     011C    _rand16
     011C    _rand16_start
     013C    _pal_clear
     013C    _pal_clear_start
     014B    _pal_select
     014B    _pal_select_start
     0153    _pal_bright
     0153    _pal_bright_start
     015B    _pal_col
     015B    _pal_col_start
     0170    _pal_copy
     0170    _pal_copy_start
     017C    _pal_custom
     017C    _pal_custom_start
     0196    _draw_tile
     0196    _draw_tile_start
     01A4    _draw_tile_key
     01A4    _draw_tile_key_start
     01B2    _draw_image
     01B2    _draw_image_start
     01BE    _draw_image_extra
     01BE    _draw_image_extra_start
     01CF    _clear_screen
     01CF    _clear_screen_start
     01D7    _swap_screen
     01D7    _swap_screen_start
     01DA    _select_image
     01DA    _select_image_start
     01E2    _color_key
     01E2    _color_key_start
     01EA    _set_sprite
     01EA    _set_sprite_start
     0214    _sprites_start
     0214    _sprites_start_start
     0217    _sprites_stop
     0217    _sprites_stop_start
     021A    _time
     021A    _time_start
     0226    _delay
     0226    _delay_start

Hexadecimal

Area                               Addr   Size   Decimal Bytes (Attributes)
--------------------------------   ----   ----   ------- ----- ------------
_DATA                              0237   0002 =      2. bytes (REL,CON)

      Value  Global
   --------  --------------------------------
     0237    _heap_top







Hexadecimal

Area                               Addr   Size   Decimal Bytes (Attributes)
--------------------------------   ----   ----   ------- ----- ------------
_HEAP                              023A   0000 =      0. bytes (REL,CON)

      Value  Global
   --------  --------------------------------
     023A    _HEAP_start
MODULES
	FILE _temp_\out.o
		NAME main
	FILE ..\evosdk\crt0.o
	FILE ..\evosdk\evo.o
		NAME evo
USERBASEDEF
	_CODE = 0x0006
	_DATA = 0x0000
